:10000000F01F0010253500002135000021350000CB
:1000100021350000213500002135000000000000DE
:10002000000000000000000000000000213500007A
:1000300021350000000000002135000051130000B0
:10004000FD100000FD100000FD100000FD1000007C
:10005000FD100000FD100000FD100000FD1000006C
:10006000FD100000FD100000FD100000FD1000005C
:10007000FD1000001D3500001D3500001D3500007D
:10008000091400002114000039140000511400006C
:100090001D350000311500001D3500001D35000024
:1000A0001D3500001D3500001D3500001D35000008
:1000B0001D3500001D3500001D3500001D350000F8
:1000C00008B500230B60036000F096FD08BD08B57D
:1000D0000A20002101F038F908BD000038B50C4BAA
:1000E0000D1C041C19680B4803F050FA212103F081
:1000F0004DFA011C012001F0D7F9012001F0B4F9FB
:10010000291C201C02F084FD012001F0BDF938BD3E
:1001100078800440001BB70008B50A4B0A481968EC
:1001200003F034FA212103F031FA011C012001F01F
:10013000BBF9012001F098F902F0ECFC012001F07C
:10014000A3F908BD78800440001BB70013B59620C2
:10015000000201F02BFA18480D210C2200F02CFCB3
:1001600000F06AFB15480021032200F099FC00F022
:100170006DFBFFF7D1FF1248124901F0FFFB00248D
:1001800001F0BEFA002802D000F0E0FE00240A20B0
:1001900001F00AF9684601A9FFF792FF009B002BC6
:1001A00003D1094B01349C42EADDFFF7B5FF074854
:1001B00001F0E4FB13BDC0464E3900005437000087
:1001C000633700006E3700006F17000075370000BE
:1001D00007B5044B04490093044A054B01F0D9FBD1
:1001E00007BDC04691370000803700006E37000021
:1001F0008937000070B50D1C161C041C00F01CFB98
:100200000B480D210C2200F0D7FB281CA1B20022C4
:1002100000F046FC07480321062200F0CDFB301C0D
:100220000121092200F03CFC00F010FB70BDC0462B
:100230004E3900000938000038B50D1C041C00F0D0
:10024000DAFA2A1C0120211CFFF7D4FF034B0022FD
:100250005A60034A943212689A6038BD281300101D
:100260008C04001010B588B0041C6846FFF7B0FF7E
:1002700069466A46201CFFF7BDFF08B010BD0000AC
:1002800073B518200021FFF729FF00243B4E012001
:1002900001F0FAF83A4D9835002C01D0002000E02A
:1002A0000620012101F050F8684601A9FFF708FF78
:1002B000009B002B21D1002CF0D12B68002B0DD0FE
:1002C000304B00941A6811321A6004E002F0CCFB43
:1002D000009B01330093009B102BF7DD2A4BF6188F
:1002E000DED518200021FFF7F9FE254B94331C685A
:1002F00063425C4100F074FACEE7002C03D0182B67
:10030000C5D100F0ABFA009B182B1BD1019BC22B6F
:1003100008D11E4B1A6801321A60022A0BD1002242
:100320001A6008E0832B06D10020FFF79BFFFFF740
:10033000F3FEFFF7CCFE019B732B01D1FFF706FF05
:1003400000230193124B1348196803F01FF9212170
:1003500003F01CF9011C012001F0A6F8012001F0B6
:1003600083F80098019902F053FC054B94331B6805
:10037000002B8AD100F034FA012487E720BF020065
:100380008C040010C00200100CFEFFFF7001001072
:1003900078800440001BB70013B501F069FB00F042
:1003A000F7FB00F05BFA00F0DDFD3C24201CFFF7BA
:1003B00059FF013C1E2000F0F7FF022CF6D102F09D
:1003C00075FA1E2300930C2301930E480E4B0F4920
:1003D0000F4A02F025FB00200421012200F0DEFD7F
:1003E0000020021C042100F027FE0020052101222C
:1003F00000F0D4FD00200521021C00F01DFEFFF7D7
:100400003FFFC046E9340000C0020010C1000000F8
:100410003902000000B500E001300378202BFBD04A
:1004200000BD00B5031C303BDAB2092A01D8181C04
:1004300008E020231843031C613B5738052B01D9E2
:100440000120404200BD70B50E1CFFF7E3FF002500
:10045000041C06E0FFF7E5FF002805DB2D0105433E
:10046000013420780028F5D13560201C70BD0000D3
:1004700070B5054E051C0E24013C295D301C01F0B1
:100480007DFA002CF8D170BD9437000000B50E2322
:10049000013BC25C002A03D1002BF9D1012000E00E
:1004A000002000BDF8B500240E2703231C4221D1F3
:1004B0003E1C66432B4D7019FFF7E8FF002815D04E
:1004C000601C78434019FFF7E1FF00280ED0301C74
:1004D0001C304019FFF7DAFF002807D02A367019C0
:1004E000FFF7D4FF002801D004340DE01E48211C82
:1004F00001F044FA381C60431A4B0134C018FFF76E
:10050000B7FF1A4801F03AFAFF2CCEDD184801F087
:1005100035FA184C201CFFF7ABFF174D4221281C61
:1005200001F02CFA201C0E30FFF7A2FF4321281CFB
:1005300001F024FA201C1C30FFF79AFF0F4801F04D
:100540001DFA201C2A30FFF793FF281C4E2101F0D2
:1005500015FA201C3830FFF78BFF616D084801F059
:100560000DFAF8BD2805001097370000315D000036
:10057000A03700008C040010A6370000AD37000043
:10058000B337000070B50E1CFFF744FF0D25041CA7
:100590002078FFF746FF002807DB01347055013D46
:1005A000F6D2201CFFF736FF00E0002070BD0000EF
:1005B00073B5394D08682B78002B06D1374801F008
:1005C000DDF902F073F9012342E00378412B1BD1DE
:1005D000334C0230211CFFF7D5FF002851D003789F
:1005E000422B4ED1211C02300E31FFF7CBFF0028E9
:1005F00047D00378432B44D1211C02301C31FFF734
:10060000C1FF002846D13CE04D2B23D1254C0230C0
:10061000211CFFF7B7FF002833D003784E2B30D1D1
:10062000211C02300E31FFF7ADFF002829D00378DE
:10063000472B26D1023001A9FFF705FF019B002BB4
:100640001FDB2A3C63651848184901F097F900231D
:100650002B701FE001A9FFF7F6FE0378202B01D0D5
:10066000002B0ED1124E00240E250199611869430A
:100670008919FFF787FF002803D00134042CF4D137
:1006800008E002F013F908480A4901F077F9024B33
:1006900000221A7073BDC04698020010BF370000D8
:1006A0008C040010B6040010D5370000DF370000BE
:1006B00028050010E237000037B54C6824E0201C04
:1006C000FFF7A8FE01A9FFF7BEFE019B041C002B4B
:1006D0001DD0D8B2FF2B09DD00F0FCF9051C0198F4
:1006E0000012C0B200F0F6F9019003E000F0F2F958
:1006F000002501900198002802D0291CFFF7EEFC8C
:1007000023785A1E9341E4182378002BD7D137BDA4
:1007100008B5064A012113784B40137001D00449F3
:1007200000E00449044801F029F908BD79030010EC
:10073000E9370000F1370000FA37000070B5051CFA
:1007400001200821021C00F077FC0724012601206B
:100750000821002200F070FC2A1C224132400020B7
:10076000022100F069FC01200821021C00F064FC59
:10077000013CECD270BD10B50021041C0A1C022003
:1007800000F05AFC201CFFF7D9FF10BDF7B501237C
:1007900000930023019372B66C46061C02AF01CC95
:1007A00050235B421843C0B2FFF7E5FF0020FFF77C
:1007B000E2FF1020FFF7DFFFE020FFF7DCFF00255E
:1007C00002200021012200F037FC705D0135FFF7A7
:1007D000B5FF842DF4D18436BC42E0D162B6F7BDBA
:1007E00008B5AC20FFF7C7FFAE20FFF7C4FFA52078
:1007F000FFF7C1FF08BD08B5AF20FFF7BCFFA4207D
:10080000FFF7B9FF08BD08B5AE20FFF7B4FF08BD7C
:1008100010B5041CF820FFF7AEFF201CFFF7ABFF5C
:1008200010BD10B5041C8120FFF7A5FF3F2020401C
:10083000FFF7A1FF10BD000008B584220248002187
:10084000520001F0D3F808BD8103001008B502483A
:10085000FFF79CFF08BDC0468103001008B50120CA
:10086000021C082100F09AFB0120021C082100F064
:10087000E3FB00200221012200F090FB0020022176
:10088000012200F0D9FB02200021012200F086FBAA
:1008900002200021012200F0CFFB022006210122CC
:1008A00000F07CFB02200621012200F0C5FB0320A2
:1008B000011C012200F072FB0320011C012200F048
:1008C000BBFB0320011C002200F0B6FB0220062126
:1008D000002200F0B1FB06210122022000F0ACFB57
:1008E000FFF7AAFFFFF7B2FFA220FFF744FFA02007
:1008F000FFF741FFC020FFF73EFF0020FFF788FF12
:100900000A2000F051FD4020FFF735FF2C20FFF7B3
:1009100032FF322000F048FD2E20FFF72CFF32205E
:1009200000F042FD2F20FFF726FF0A2000F03CFDDB
:100930002520FFF720FFAF20FFF71DFFA420FFF7C2
:100940001AFF0020FFF76DFF08BD000000B50F295A
:100950000ED883280CD8CB08842253430722C01812
:100960001140044B80220A41111C1A5C1143195496
:1009700000BDC04681030010F0B55B18DBB216E085
:100980008425CC086C4307270F40802504193D417E
:10099000EFB2A6189C4605E0064BE5182B7801340B
:1009A0003B432B70B442F7DB01316346C9B2994235
:1009B000E6D3F0BD8103001000B5084B1860084B6A
:1009C0001970084B20211A70074B1970074BD1087A
:1009D0001970500701D00131197000BD7C0300105F
:1009E000890400108B0400108A040010800300109A
:1009F000F0B5284B89B01B780024C01A264B06920C
:100A000005911B68221C04E002310C190132A4B2CA
:100A1000D2B2195D8242F7DB1B195B780391029316
:100A200000222CE000994B4303999A198A4214DA68
:100A3000194A0025126892191219D3189B78049349
:100A40000123049AAB40134204D07919C9B2079824
:100A5000FFF77CFF0135082DF2D101360837F6B2D9
:100A6000FFB206E00099059A069F8B18DBB20026BC
:100A700007930A490B789E42D4D3019A013201921E
:100A80006B461B79029900938B42EBD309B0081C8B
:100A9000F0BDC0468A0400107C03001080030010E3
:100AA000F7B5171C061C0D1C00F0C0FF80B20190AA
:100AB0000024FFB208E0305DE9B23A1CFFF798FF6E
:100AC00001302D18ADB20134019AA3B29342F2D392
:100AD000F7BD000000B50F23020918408000031F76
:100AE00000D52833002B0EDB511E032088428041A5
:100AF0004042002807D1242B06DC04218A1A03492E
:100B0000CB18985C00E0002000BDC046513D0000BD
:100B100010B5041C211C144800F0B2FA211C134823
:100B200000F0AEFA211C124800F0AAFA211C11486C
:100B300000F0A6FA211C104800F0A2FA211C0F4870
:100B400000F09EFA211C0E4800F09AFA211C0D4874
:100B500000F096FA211C0C4800F092FA0B48211C78
:100B600000F08EFA10BDC0462040044024400440EE
:100B7000284004402C400440384004403C4004409D
:100B80004040044044400440484004404C4004403D
:100B9000F8B51020FFF7BCFF094C271C1437257847
:100BA0006678281C311C002200F0F8F90234281C59
:100BB000311C012200F040FABC42F0D1F8BDC04621
:100BC000793D0000F8B50B4C271C14372578667862
:100BD000281C311C012200F0E1F90234281C311CD0
:100BE000002200F029FABC42F0D10020FFF790FF6C
:100BF000F8BDC046793D0000F0B589B000240490EE
:100C00000591FFF7C5FF02200721012206940794F2
:100C100000F0C4F902200721221C00F00DFA201C6C
:100C20000B2100F0DFF9A04202D118230693012422
:100C30000021264D03916A782F78111C0192381CEF
:100C4000012200F0ABF9381C0199002200F0F4F900
:100C500003231F4E029314E03078717800F0C2F93C
:100C6000002807D103991B4AA3008A5C1833694600
:100C70005A500134029A039B013A013302920393C2
:100C8000023EE30F00210122A2424B41DBB28B4224
:100C900002D0029B8B42DFDA381C0199002200F05F
:100CA0007DF90199381C012200F0C6F90A49023584
:100CB0008D42C0D1201E06D0069B049A0599136070
:100CC000079B01200B6009B0F0BDC046793D0000D4
:100CD0004F3D0000513D00008D3D000000B50A4B26
:100CE00000211960094B01221A6019601A60196805
:100CF0001142FCD0064B01221A60064B8022196873
:100D000052020A431A6000BD70800440748004409F
:100D1000788004408080044008B500F031F90C4B25
:100D200003201A68120B12031A600A4B1A68120B7E
:100D300012031A60084B1A68120B12031A60074B51
:100D40001A68120B12031A60FFF7C8FF08BDC046ED
:100D5000008000500080015000800250008003504D
:100D600070B5124A1249134800F008FE124C13489D
:100D7000211C00F003FE201C00F000FE104E114D5F
:100D800000242B196159DA68301C0B4B143400F025
:100D9000F5FD642CF5D10C4800F0F0FD00F020FBCF
:100DA000011C0A4800F0EAFD70BDC046893700000A
:100DB0006E3700008D3D0000FF3D0000A13D0000AA
:100DC000BA3D000000000010C53D0000EC3D0000F1
:100DD000F0B53C4B8BB01D78002D3AD03A4B0290C9
:100DE0001B6801209B685DE001342378202BFBD039
:100DF000002B3AD0B30008336A469C500136FF2DD1
:100E000001D135E001342378202B01D0002BF9D11A
:100E1000202B02D1002323700134012E1BD12A4F35
:100E20002A4B06223B6001923D1C09E02B68029888
:100E3000196800F00EFE002808D02B6814332B60D0
:100E4000019B013B0193002BF0D132E03B681D79FF
:100E500001E0041C2E1C2378002B06D0002307225F
:100E6000B2425B41DBB2002BBFD1002E1CD000E0B0
:100E70000025154C022E05D10398154900F0E9FD17
:100E8000002801D0AE420AD823681248D96800F081
:100E900075FD23681048196900F070FD04E02368AF
:100EA000F0B29B6802A99847064B1B78002B07D12C
:100EB00003E00198011CFFF753FF084800F05EFDB6
:100EC0000BB0F0BD98020010A0020010000000104E
:100ED000F93D0000FB3D0000DA370000023E000053
:100EE00038B5041C154D0A2808D002D808281CD192
:100EF00010E00D2802D07F2817D10BE02B680022CC
:100F00001A700F4800F03AFD0E4C201CFFF760FFEE
:100F10002C6012E02A680B4B9A420ED90A48211C19
:100F200000F02CFD2B68013B06E00748211C00F077
:100F300025FD2B681C7001332B6038BD9C0200100E
:100F4000FF3D0000980100100E3E000008B503E0D0
:100F500000F0B4FBFFF7C4FF00F0D2FB0028F7D18C
:100F600008BD000008B5034A034B04481A6000F0AE
:100F700005FD08BD980100109C020010023E000013
:100F8000044B40211A680A431A60034B01221A706D
:100F90007047C04680800440A402001070B50E4B1C
:100FA000061C1B780D1C141C002B01D1FFF7E8FF59
:100FB000013E022E03D8094BB600F35800E0084B5F
:100FC0001A68012C03D1AC4014431C6003E00124D7
:100FD000AC40A2431A6070BDA40200107C3E000029
:100FE0000080005038B50F4B051C1B780C1C002BE3
:100FF00001D1FFF7C5FF0020032D11D8281C0123C4
:1010000002F0B0FA02040608074A04E0074A02E0C8
:10101000074A00E0074A1068A3401840431E984161
:1010200038BDC046A4020010FC3F0050FC3F0150F8
:10103000FC3F0250FC3F035070B50E4B061C1B7862
:101040000D1C141C002B01D1FFF79AFF013E022E4C
:1010500003D8094BB600F35800E0084B1A68012C7E
:1010600003D1AC4014431C6003E00124AC40A24314
:101070001A6070BDA4020010883E0000FC3F0050C2
:1010800038B5084B041C1B780D1C002B01D1FFF751
:1010900077FF236818229343236023681D4325604C
:1010A00038BDC046A40200101F2342091840012386
:1010B0008340181C014B9200D050704700E100E0C3
:1010C000054B3F221A60054B01221A60044B402158
:1010D0001A688A431A60704724800440D88004400C
:1010E0003882044008B5044B40211A688A431A60CC
:1010F000FFF7E6FF08BDC0463882044008B503206C
:10110000FFF7ECFD094B012252421A60084A1268AF
:10111000002A00D01A60074B1A6801321A60064A8A
:1011200000231360054A1360C04608BD08820440CE
:101130000C820440A802001004C000403CC00040E3
:1011400008B5FFF73FFD0A480021FFF799FF09485E
:101150000021FFF795FF08480021FFF791FF07489E
:101160000021FFF78DFF06480021FFF789FF08BD2A
:101170000840044000400440AC4004401440044097
:101180001C400440F7B50190FFF7DAFF574B019977
:101190001A68574B1A60002901D0564B00E0564B95
:1011A000564A04211360564B564C1A68564D0A4352
:1011B0001A60019A002A54D0544B0027544E1F60E5
:1011C000544B301C1F60391CFFF75AFF381C092193
:1011D0003A1CFFF7E3FE381C09213A1CFFF72CFFED
:1011E0004D4B802219680320114319603368072191
:1011F0008B433360336802210B43019933604B000A
:101200005B1899015B1801999B005B1843490B60BF
:10121000434B196801431960424B43491868014028
:101220001960196809200A431A60FFF73DFF226818
:1012300080239B001A43226001213C4A49421160ED
:101240002A68324913432B60394B02221A60394B0A
:1012500001221A601F601A6018681042FCD0012336
:101260000B600720FFF720FF0820FFF71DFF0A2073
:10127000FFF71AFF0C20FFF717FF0B20FFF714FFF3
:10128000236880229343236022682B4B1340236002
:1012900022682A4B134023602268294B13402360A5
:1012A0002268284B13402360019B002B03D10122AD
:1012B0001E4B52421A602B68802213432B602A680F
:1012C00080235B0013432B602A688023DB001343D9
:1012D0002B602A6880235B0113432B602A688023DC
:1012E0001B0113432B6030BFF7BDC046388204405A
:1012F00034820440BF180000FF1800003082044010
:1013000010ED00E0008204400482044004C000406C
:1013100064400440044001408080044018C0004004
:1013200014C000403CC000400FF0FFFF08820440A2
:101330007080044074800440FFFEFFFFFFFBFFFF4E
:10134000FFEFFFFFFFF7FFFF08B5FFF71BFF08BD2B
:1013500000B5064B1A6801321A601B68013303D1CD
:10136000034B1A6801321A6000BDC046B00200107B
:10137000AC02001000B5074B98420AD8064A002379
:101380001360064A01381060054A1360054B0722B6
:101390001A6000BDFFFFFF00B002001014E000E083
:1013A00018E000E010E000E000B50C4A13680028E7
:1013B00000D10120C1438B4204D809E01168814269
:1013C000FCD301E0591C081811689942F6D203E0D9
:1013D0001168C91A8142FBD300BDC046B00200109B
:1013E00010B5064BFA211868054B89001C6802F0FD
:1013F000CDF8044B5C43201810BDC046B00200106D
:10140000AC02001037894100034B01221A60034BE4
:101410001A6801321A60704700C00040B402001020
:10142000034B01221A60034B1A6801321A6070479D
:1014300000000140B8020010034B01221A60034B68
:101440001A6801321A60704700400140BC02001067
:10145000034B01221A60034B1A6801321A6070476D
:1014600000800140C002001000B5002803D1044BE9
:1014700001221A6003E0012801D1024B186000BD6F
:10148000044001400480014000B5002802D1044B13
:10149000186004E0012802D1024B00221A6000BD4E
:1014A000044001400480014010B5041C002906D10D
:1014B000164B96201968C00002F068F8011C002C39
:1014C0000FD1134B80221868920002431A60114B0F
:1014D00003221C60104B1960104B1A608022D2024C
:1014E00011E0012C11D10A4B80221868D20002436E
:1014F0001A600B4B00221A600A4B032219600A4B38
:101500001A6080221203094B1A6010BD78800440D3
:1015100080800440BC02001018400140144001408B
:10152000C0020010188001401480014000E100E07A
:1015300008B5184B1A680E231340062B0DD1164B15
:101540009E221B68DBB2134204D0144A5360144B32
:101550001B681EE0D9071CD501E0042B05D1104BF8
:101560001868C0B200F0BBF813E00C2B06D10B4B8F
:101570008022596852000A435A600AE0022B08D1BF
:10158000054B1A68054B910601D5002200E00122A7
:101590009A6008BD0880004014800040C40200101A
:1015A0000080004000487047C402001070B52B4C0A
:1015B0002B4B80229203DA6700219022061C201C0C
:1015C00000F014FA0023A36000F072F8254B072501
:1015D0001A68254CAA431A60196801221143196040
:1015E000224B1968A9431960196811431960204BEF
:1015F000802118684901014319601E4B1E481A607A
:101600008322226019681D4B1B68584301F0BEFFFE
:10161000311C000901F0BAFF1949030A194A0B608D
:10162000C0B2032310602360174B1D60174B18686E
:1016300060201C680440602CFBD101E0146800E0CD
:1016400001201C680442F9D1044B01221A70104B8E
:10165000802292031A6005230B6070BDC402001043
:1016600004E100E0A44004400C800040A840044095
:101670008080044098800440001BB70078800440BC
:10168000048000400080004008800040148000403A
:1016900000E100E000B5044A202311681942FCD0A3
:1016A000024B186000BDC04614800040008000401E
:1016B00008B5FFF777FF0023437308BD08B5FFF7B0
:1016C00071FFC27B031C8218107CDA7B7F21013200
:1016D0000A40DA735A7B013AD2B25A7308BD10B588
:1016E000041CFFF75FFF837B7F22C3181C74837B7E
:1016F000013313408373437B0133DBB2437310BD6B
:1017000008B5FFF74FFF407B431E984108BD30B539
:10171000002402E00570013401301D5D002DF9D177
:10172000121B131C02E00170013B0130002BFADC9C
:10173000D043C0170240A01830BDF8B5051C0F1CDF
:101740001E1C541E092B01D800240FE0181C0A216E
:1017500001F01CFF221C031C391C281CFFF7EDFFA5
:10176000041C2D1805E02F7001340135013A002AC0
:10177000F9DC301C0A2101F04DFF30312970601C6A
:10178000F8BDF8B50C1CD9175F18061C4F40551E44
:10179000092F12D9381C0A21002B03DA01F0F6FEBA
:1017A000434202E001F0F2FE031C211C2A1C301C03
:1017B000FFF7E7FF041C351813E0002B00DA951E35
:1017C000002201E0B4540132A91A0029FADCEC43EA
:1017D000E4172C403519002B03DA2D232B7001342C
:1017E0000135381C0A2101F015FF30312970601CC9
:1017F000F8BD73B5069E041C1D1C3009531E00283D
:101800000AD000901A1C201C2B1CFFF7F2FF241892
:1018100005E0217001300134013A002AF9DC0F2380
:101820001E40092E01D8303604E0002D01D0373695
:1018300000E057362670013076BDF0B585B0041C47
:101840000F1C002801D00021017000256BE0252924
:1018500003D021700132013405E05178252904D1EB
:1018600021700232013401355DE0302903D00132AC
:101870000292202101E002320292029E9C463278BE
:101880002D3A50424241B6180296002205E00A2342
:101890005A438218303AD2B201363078031C303BBA
:1018A000092BF4D90296AE186346BE4201D97A1BC1
:1018B000D2B269280ED006D863282CD0642809D06B
:1018C00058283ED119E075280AD078280FD07328FF
:1018D00037D11AE01E1D201C1B68FFF752FF04E0E1
:1018E0001E1D201C1B68FFF728FF331C17E01E1D60
:1018F0001B68201C0093002304E01E1D1B68201C95
:1019000000930123FFF775FFEFE71E1D201C1B68E6
:10191000FFF7FDFEE9E71A68012022700433029AFE
:10192000241801322D181178BD4201D200298ED120
:101930000023BD4201D2237005E0013C2370013D2C
:1019400001E001256D4205B0281CF0BD10B50C1C4E
:10195000131C6421221CFFF770FF10BD00B5031C8F
:101960009BB00A1C01A8191CFFF7F0FF632800DDDB
:10197000FEE701A800F09CF81BB000BD0FB407B54E
:1019800004A901C90191FFF7E9FF03B008BC04B045
:1019900018470EB403B503AA02CA0192FFF7D6FF97
:1019A00002B008BC03B0184770B50323041C1842EA
:1019B00005D10D1C041C194201D1934201D300230F
:1019C00011E0131C40CD043B40C4032BFAD8141F74
:1019D000A4080134A400032309191A400419EEE7EE
:1019E000CD5CE55401339342FAD170BD30B50B04A0
:1019F0000D061D430D430B021D430323041C93429C
:101A00000DD218420BD1131C043B20C4032BFBD86E
:101A1000141FA4080134A40003231A40041900234E
:101A200001E0E15401339342FBD130BD00B5002306
:101A300000E00133C25C002AFBD1181C00BD00B5D8
:101A4000031C01E0013101330A781A70002AF9D130
:101A500000BD00B502E00130002B06D00A78037803
:101A600001319342F7D0981A00E0181C00BD000025
:101A700008B5FFF751F90B48FFF77CFCFFF780FA38
:101A8000FFF730FB96200002FFF790FDFEF7E6FE21
:101A9000FEF7D2FE044A0548111CFFF76FFFFFF75F
:101AA00061FA08BDE02E0000FF3D0000943E0000FA
:101AB00010B5041C02E00134FFF7ECFD207800288B
:101AC000F9D110BD00B50B4B984201DD0A4BC0188F
:101AD0000A4A8310D35C03220240082152008A1A6A
:101AE00093401A1CC0239B001A40054B1B5C101C22
:101AF000184300BDFF17000000F8FFFFC2560000AA
:101B0000C23E000008B54018511A013101F0EEFD47
:101B100008BD08B5801889189A1A0132FFF744FFEA
:101B200008BD000030B5B14B87B0D96EB04D4A1E2C
:101B300091416A46D175A96A1A1CC806400F01383E
:101B4000062807D801F00EFD040C1F1217191C00FF
:101B5000022409E05A6E16329200D3581C1C15E07C
:101B60005B6E16339B00D45800230FE09B6DD46D41
:101B7000A3420ADC0AE0022403E00C24032305E06C
:101B80000D24231C02E00D24EEE70D242C614811E6
:101B90001F2800D922E16A461732944901F0ECFC73
:101BA0002000220028002A002D002F0038004000CD
:101BB0004400490051005F0067006F007700850016
:101BC0009300A200B400C300D500D300E300E600F8
:101BD000E900F100010105010F01110113011901D3
:101BE000081C00E08348191C221CFFF78BFFF5E05E
:101BF0008148F8E70A1C0E3203E07E4809E00A1C1F
:101C00001C32081C111C1A1C231C01F0FDF8E5E015
:101C10007948011C0E391A1C231CFFF77AFFDDE0FE
:101C20007448011C0E31EEE70A1C1C32081C111C02
:101C3000F1E70A6E1020002A00D00A200A1C0E329A
:101C400006E00A6E1020002A00D00A200A1C1C326E
:101C500000946C46173402900194081C51E0012056
:101C60001070086E1022002844D00A2242E00A6E4A
:101C70001020002A00D00A200A1C0E320EE001209B
:101C80001070086E1022002855D00A2253E00A6E08
:101C90001020002A00D00A200A1C1C3200946C4636
:101CA000173402900194081C78E00A6E1021002A73
:101CB00000D00A21504A68461730019002910094E2
:101CC000101C111C1DE00A6E1020002A00D00A20F2
:101CD000494A00946C46111C173402901C39019437
:101CE000101C0EE0096E012010701022002900D097
:101CF0000A22414968461730019002920094081C5C
:101D0000002201F08BF869E00A6E1020002A00D052
:101D10000A20394A00946C46111C173402901C3971
:101D20000194101C3AE0096E012010701022002965
:101D300000D00A2230496846173001900292009480
:101D4000081C00222AE0012010700A6E1021002ACF
:101D500000D00A21284A6846173001900291009469
:101D6000101C00211AE0009222481CE00092224838
:101D700019E00A6E1020002A00D00A200A1C1C322A
:101D800006E00A6E1020002A00D00A200A1C0E323B
:101D900000946C46173402900194002001F067F81B
:101DA0001CE00092081C002104E00D1C1C35081CDE
:101DB0000092291C1A1C231C01F0B4F80EE0081C28
:101DC00002E00C4800E00C48191C221C01F0C3F88A
:101DD00004E0081C221C191C01F0C8F86B46DA7DCF
:101DE000024B07B00120DA6630BDC0468C040010FB
:101DF000281300109A040010A804001010B506491A
:101E00000B1C88331A68141C1E34A4006050013265
:101E100003210A401A6010BD8C040010054B0320FA
:101E2000191C88310A68013A02400A601E32920089
:101E3000D05870478C040010F8B5114D2C1C8C3410
:101E400020680130FFF73EFE0E4B0122D8629F6AE8
:101E5000AB6E061C02409A4210D1830703D420685F
:101E60000230FFF7CBFFFF239B001E40B601BF10DF
:101E7000044B8C35374301222F60DA600220F8BD15
:101E80008C0400102813001030B50C4B0C489A6AD3
:101E9000031C8C331C68D3059B0E910500D5403B79
:101EA000856E921001210A40AA4204D1E3188C30B9
:101EB0000360024BD960012030BDC04628130010DA
:101EC0008C04001008B5084B5A1CD07F9A1CD27F96
:101ED000000112021043DA7F0333DB7F10431B0340
:101EE0001843FFF78BFF08BD8C04001038B5FFF7CF
:101EF00095FF064903230F22051C5C18154001338A
:101F000025770011072BF7D138BDC0468C0400108F
:101F100008B5FFF783FF034B01228C331860024B97
:101F2000DA6008BD8C0400102813001010B5064CB0
:101F3000A36E002B06D0FFF771FF044B8C340122F7
:101F40002060DA6010BDC0468C0400102813001019
:101F500010B5064CA36E002B06D1FFF75FFF044BB4
:101F60008C3401222060DA6010BDC0468C04001061
:101F70002813001008B5124B1B68002B00D098479F
:101F8000104B5A69002A15DD012A07D1DA69002AA7
:101F900004D09A610022DA610A225A615B69032245
:101FA000191C91430A1E02D0074A0121D166054A35
:101FB000013B5361044B90331A68024B5A6208BDCF
:101FC00054030010281300108C04001000B5064BB9
:101FD0005A69002A07DD9A690F21044B1140D9770D
:101FE00012110133DA7700BD281300108C040010A1
:101FF000044B597F9A7F090112020A43197F0A4351
:102000005A6770478C04001030B50B1C093B012B3C
:102010000FD8084A00239C18257FC45CA54205D030
:10202000054B08395A681143596002E001330E2B01
:10203000F1D130BD8C0400102813001000B5082920
:102040000DD0192911D1427808231A4202D000225A
:10205000027002E00F2303700723437005E00023A2
:102060001A1CC25401330E2BFBD100BD10B50E4B10
:10207000596F002802D00F22914301430E244C4394
:1020800059679C33E418094B1B68292B02D0201C8C
:10209000FFF7D4FF044A0023E05C99180133087766
:1020A0000E2BF9D110BDC0468C040010281300106F
:1020B00070B5124B0F225C6F944304435C67104B66
:1020C0001B68292B01D0082C17D00E2565430D4E17
:1020D000211CAD19281CFFF797FF9C3E00239A197D
:1020E000127FEA5401330E2BF9D1054B1B68292BC3
:1020F00003D0281C211CFFF7A1FF70BD8C04001029
:10210000281300102805001038B5104B104D1B681F
:10211000292B02D06B6F082B17D0696F0E244C430C
:102120009C356419201CFFF76FFF9C3D00235A1952
:10213000127FE25401330E2BF9D1044B1B68292B7B
:1021400003D0696F201CFFF779FF38BD28130010FA
:102150008C04001010B50D4C631CD87FA31CDB7FD2
:1021600000011B021843E37F1843E31CDB7F1B03C2
:102170001843FFF7A7FC0F23021C1A402277021115
:10218000134000126377A07710BDC0468C04001086
:10219000044B5A6E16329200D258121A51424A41DA
:1021A000DA6670478C04001000B5064B5A6E163282
:1021B0009200D1580139D150002901DA0D21D150B6
:1021C00000BDC0468C04001000B5064B5A6E163296
:1021D0009200D1580131D1500E2901D10021D150A6
:1021E00000BDC0468C04001000B5094B5A6E163273
:1021F0009200D2580D2A03D11A1C2932127805E018
:102200009A18507F117F0001021C0A435A6500BDD5
:102210008C04001010B5084B0F245A6E1632920031
:10222000D1585A6D58181440013104770D2902DC39
:102230005B1812111A7710BD8C04001030B50F4BCB
:102240005A6E596D16329200D2580D2A07D11C1CB5
:1022500029342478F02008402043586507E0981876
:10226000447F057F24012C435C650B114377034BAE
:102270009A180F231940117730BDC0468C04001006
:1022800008B504480022011C1C390D23FFF741FC4E
:1022900008BDC046C404001008B504480022011C53
:1022A0001C310D23FFF735FC08BDC046A804001003
:1022B00008B504480022011C1C310D2300F0A4FDC8
:1022C00008BDC046A804001008B504480022011C3F
:1022D0000E390D23FFF71DFC08BDC046B6040010E3
:1022E00008B504480022011C0E310D23FFF711FC34
:1022F00008BDC046A804001008B504480022011C0F
:102300000E310D2300F080FD08BDC046A80400106A
:102310000C4A0023111C46310B70111C47310B7005
:10232000111C48310B70111C49310B70111C4A31C2
:102330000B70111C4B310B70111C4C314D320B705A
:10234000137070478C04001000B5074A011C042369
:1023500000208A1804E0D11846310978400008436B
:10236000013BF8D200BDC0468C04001030B5074ACE
:1023700000238918012206E0CC18051C46341540BC
:10238000257040100133042BF6D130BD8C040010B1
:1023900038B50020FFF7D8FF084C051C0021207F2E
:1023A000FFF7E4FF25770420FFF7CEFF0421051C8B
:1023B000607FFFF7DBFF657738BDC0468C040010F7
:1023C00010B50020FFF7C0FF034C20770420FFF773
:1023D000BBFF607710BDC0468C04001010B5054CE3
:1023E0000021207FFFF7C2FF607F0421FFF7BEFFBF
:1023F00010BDC0468C04001010B5094C231C8C3352
:1024000018680130FFF75EFB064B021CD8620F23F1
:102410001A4022770211134000126377A07710BD93
:102420008C0400102813001010B5094C0021201C4A
:102430000D22FFF767FB201C0E3000210D22FFF755
:1024400061FB201C1C3000210D22FFF75BFB10BD3F
:102450008C04001010B50C4B00211A1C187F1C783E
:1024600001312043187701330E29F7D1936E002BE9
:1024700008D0064B1B690D2B04D1137F111C293189
:102480000B70537310BDC0468C040010281300104D
:1024900010B50C4B00211A1C1C7F1878013120400C
:1024A000187701330E29F7D1936E002B08D0064B15
:1024B0001B690D2B04D1137F111C29310B70537331
:1024C00010BDC0468C040010281300107FB50023F7
:1024D0000C4A0D251C1C1118097F01306E469955B8
:1024E000C60F8542664176420133111C30400E2BE7
:1024F000F1D100236C46185DCA18013310770E2BFA
:10250000F8D17FBD8C04001010B5074B5A6E1632FF
:102510009200D1585C1801392077D150002901DA96
:102520000D21D15010BDC0468C040010034A002379
:10253000111C943198320B60136070478C040010AA
:10254000034B012194331A684A401A607047C04611
:102550008C040010044A002313678C321360034B71
:102560000122DA607047C0468C0400102813001066
:1025700008B59A4B0F20996A994A8B101840891117
:10258000013852560E2800D9C1E000F0EBFF0811C7
:102590001A2327C02EC0C037C0C0C03B3F00002A4E
:1025A00000DAB4E08F4B9A18403200239371A9E00F
:1025B000002A00DAABE08B4B01209A184032907170
:1025C000A4E0002A00DAA2E0864B9A184032927901
:1025D000DA6697E0081CFFF797FF93E0002A00DA1D
:1025E00095E0101CFFF7D4FD8CE0002A00DA8EE0A5
:1025F0007C4B596E16318900CA5083E0081CFFF7E6
:1026000057FD7FE0081CFFF731FD7BE0002A00DA70
:102610007DE0101CFFF75AFF74E0724B01209833E5
:10262000186073E0FFF7E0FD6CE0FFF793FF69E0EF
:10263000FFF726FE66E0FFF7EDFD63E0694B002241
:102640005A665FE0FFF728FE5CE0FFF7F7FD59E010
:10265000644B0120586659E0FFF72AFE52E0FFF76D
:10266000CBFE022052E0FFF72FFE4BE0FFF72AFCE3
:1026700048E0FFF735FE45E0FFF7D6FE42E0FFF702
:1026800035FC3FE0FFF738FE3CE0FFF79FFC39E008
:10269000544B00221A6635E0FFF7AAFC32E0514B9A
:1026A0000120186632E0FFF741FF2BE0FFF72CFD19
:1026B00028E0FFF745FF25E0FFF74CFD22E0FFF79C
:1026C0008DFE1FE0FFF732FC1CE0FFF7C3FE19E0B0
:1026D000FFF776FE16E0FFF73BFC13E0FFF7D8FEAE
:1026E00010E0FFF715FE0DE0FFF744FC0AE0FFF7EE
:1026F0005BFD07E0FFF74CFE04E0FFF765FD01E03E
:10270000FFF706FC012001E00120404208BD982BA4
:10271000BED03EDC382B9BD01DDC1C2B00D187E7C4
:102720000CDC0C2B00D178E702DC002BEAD0EBE7C5
:10273000162B00D176E7182BE6D176E7282B00D1AF
:102740007CE702DC262BDFD175E72C2B00D179E763
:10275000362BD9D179E7662B00D18AE70CDC4C2BDC
:1027600000D17CE702DC3C2BCED175E7562B00D1A3
:1027700079E75C2BC8D179E76C2B00D17FE702DCCD
:10278000682BC1D178E7762B00D17BE7882BBBD1B2
:102790007BE7E62B00D19BE726DCC82B00D188E73E
:1027A0000CDCA82B00D17AE702DC9C2BACD173E7C0
:1027B000B82B00D177E7BC2BA6D177E7D62B00D179
:1027C0007DE703DCCC2B00D09EE775E7D82B00D14A
:1027D00078E7DC2B00D097E777E7C0462813001096
:1027E000C25C00008C040010F32B00D17CE70EDCEF
:1027F000EC2B00D172E703DCE82B00D084E76AE71A
:10280000F12B00D16DE7F22B00D07DE77AE7F62BB4
:1028100000D16FE703DCF52B00D075E767E7F72BF6
:1028200000D16AE7F82B00D06EE769E738B5184C9D
:10283000231C8C331868FFF745F9211CE26E903198
:10284000144B0D68A2660022E2660135DA600322AD
:1028500098620D601040251C1C1C022809D0904273
:102860000AD0012802D0FFF783FE07E0FFF7E4FA61
:1028700004E0FFF757F901E0FFF706FB002806DD4B
:10288000E368002B03D18C352B681B182B6038BDF7
:102890008C04001028130010034B0122DA660F226B
:1028A0009A775A771A7770478C04001010B5054C48
:1028B0000549201C00F01AFFFFF7EEFF01236366B5
:1028C00010BDC0468C0400109C0E000000B5074BE4
:1028D00000201B680F2B08D1054B1A78824204D1C7
:1028E0001868044B1840431E984100BD6400001056
:1028F0008C04001000FFFF0038B5164B1A1C9832EC
:102900001268002A04D0144B1D6801231D4001E009
:1029100094331D68114CA3689D4202D16268002A5D
:1029200016D0002D02D1002B0AD111E00C4B1B68F0
:10293000002B02D06168281C98470023636006E0E2
:10294000074B1B68002B02D0281C291C9847A56048
:1029500038BDC0468C04001074030010281300100A
:102960006C03001013B5002300930193244B1B68E4
:10297000002B02D0684601A998472249009B08789D
:10298000214A00280CD0002B02D00223137035E01E
:102990001378013BDBB21370002B2FD10B7009E0D1
:1029A000002B0CD11378002B28D0013BDBB2137025
:1029B000002B23D1154A1360154A13601EE01449F9
:1029C0000968581A44426041400010701148446937
:1029D000021C002C04D08B4202D10A2343610DE07B
:1029E00000290BD10A21516101999361D161084AF3
:1029F0001360064B02221960034B1A7013BDC046C8
:102A00005C03001078030010600300105C130010DA
:102A1000581300102813001008B5FFF7A3FF08BDD6
:102A200010B5094C20600948016009490A60094A4B
:102A30001360094B029A1A60084B039A1A60084AFD
:102A4000084B1A6010BDC0466C0300105C030010F8
:102A500068030010640300105803001064000010A5
:102A6000192A00005403001008B5084B084A1968D9
:102A700012688A1A1A6006D5FA2252001A60054BAB
:102A80001A6801321A60FFF737FF08BD68000010AE
:102A90005803001074030010F7B50E1C0E21051C1E
:102AA000019200F023FE1A4B03240C279E420FDDF7
:102AB00009236B7301232B7328E0301C0A2100F0DB
:102AC00009FE301C29550A2100F0AEFD0134061C18
:102AD000002E06D0E30F0022A7425341DBB29342FF
:102AE000EBD1019AA31A033B2B70621B2B1C01E054
:102AF000195D5973013BD1180229F9D10F231C1B11
:102B0000002301E0013C2B55032CFBDCF7BDC04644
:102B1000FFC99A3B38B50C4B01221A700B4B0222AD
:102B20001A700B4D0B4C08E01868884208D01B68DF
:102B30002360FFF799FFFFF715FF2B682168024A12
:102B400010780028F0D138BD780300106003001021
:102B500064030010700300104278037812011A43D6
:102B6000C37881781B010B43D01A7047F0B5224A15
:102B7000224B0F1CD45CE8235B00D35C24011C4374
:102B80001F4BE121D35C4900515C1B0185B00B4315
:102B90000293E9235B000390D55C002C02D18024D2
:102BA00007256400174E301CFFF7D6FF0299421C20
:102BB000631A802149000C1B07214D1B0398124901
:102BC00001950094FEF7E5FE00233B704125023E8F
:102BD000381CFEF72BFF3C18301CFFF7BDFF2A1CEA
:102BE000031C0A49201C0135FEF7D3FE023E462D88
:102BF000EED105B0F0BDC0468C040010D10100003C
:102C0000C301000058060010D25C0000DF5C000029
:102C100030B53D4B3D4C1A1C9432126891B0A06106
:102C2000E161002A17D118280BD1C32909D1384AEC
:102C300012680F2A05D1181C38300E21162200F018
:102C4000CFF8A369182B04D1E369332B01D100F02D
:102C500071F8FFF721FE0A2363612B4C01232D4DF0
:102C600023678C34FFF7E2FD2368AB4218D006DC03
:102C7000294A934219D0294A93422ED106E0284A84
:102C8000934208D0274A934227D117E0204B1B6874
:102C90000B2B22D10DE01E4B1B680C2B1DD108E025
:102CA0001B4B1B680F2B18D103E0194B1B68102B13
:102CB00013D1FFF721FEFDF70AFA0EE0144B1B6853
:102CC0000F2B0AD1684608A9FFF750FF164B1B6867
:102CD000002B02D0684608A99847144B1A68144B79
:102CE00010681968884205D012681A60FFF7BCFEA8
:102CF000FFF738FE044B1B6F002BB3D1FFF7FCFD31
:102D0000FFF708FF11B030BD8C040010281300102D
:102D100064000010790D00006A0C0000130D000023
:102D2000990D00006527000068030010640300107F
:102D30007003001070B5254C23681D68FFF7EAFE8C
:102D400023681A689542FCD01E68FFF7A5FD204B4A
:102D50000A22204C5A6118229A611522DA61231C3A
:102D6000903300221A60FFF797FD01232367643632
:102D7000164C194D0AE0FFF759FD23682A681968B7
:102D8000914203D01B682B60FFF76EFE23681B681F
:102D90009E42F0D10F4D18202B1C90331C6800214F
:102DA000FFF736FF0D4B60001968001900F03CFC7E
:102DB0003835011C0422281CFFF76EFE044B182234
:102DC0009A610022201CDA6170BDC04664030010C5
:102DD000281300108C04001070030010580300101A
:102DE000F0B501240DE005780B1C254006E0C65C1B
:102DF000ED0077083D43C554351C2540013BF6D511
:102E0000013A002AEFDCF0BD30B504E0845C8D5C53
:102E100085548C5401329A42F8DD30BDF7B5099DD6
:102E20000AAC2678089F2C7894461D1C002A0DD1E8
:102E300018E063465B5D4A5DD218131901920024C5
:102E4000B34201DB9B1B012443550135BD42F0DD3C
:102E50000AE0CA5C12190024B24201DB921B012471
:102E6000C2540133BB42F4DD099B1C70F7BDF7B5BA
:102E7000099E0AAC2778089D347800282FD00029B5
:102E80002AD01E1C9446002A0ED1013F18E063464A
:102E90009B5D8A5DD21A131B00240192A34201DAC2
:102EA000DB19012483550136AE42F0DD37E0CA5C00
:102EB000121B0024561C01D13A1C0124C2540133B8
:102EC000AB42F4DD2BE0D15C49420C1B211E01D04A
:102ED000E1190124C1540133AB42F4DD1FE00029A4
:102EE0001BD0181C002A06D10EE00E5C135C0130CA
:102EF000F31A1C1BE40FA842F7DD10E0CA5C013393
:102F0000141B013462425441AB42F7DD07E0D15C4F
:102F1000013349420C1B611E8C41AB42F7DD099A1B
:102F20001470F7BD70B5049D01242C70141C002989
:102F300005D10BE0065D0A5D96420BD101349C423F
:102F4000F8DD05E0815C002904D101329A42F9DD07
:102F500000232B7070BD00B503E043185B78435429
:102F600001319142F9DB0023435400BD00B504E078
:102F70008318013B1B788354013A8A42F8DC002312
:102F8000835400BDF0B5114B1A785B78825C1A400F
:102F900000D040220E4C0F49231C261C04C32C36A3
:102FA00000221A6001240A1C123117785578C75D77
:102FB0003D4202D01F6827431F60023264008A42EC
:102FC000F3D10433B342EBD10020F0BD6101001016
:102FD000F0140010AD00001030B512234B43334AFB
:102FE0000131D3188A0051181A785C78825C144237
:102FF00004D02F4A5F245218947054709A78DC7869
:10300000825C144204D02A4A7C2452185332147031
:103010001A795C79825C144204D0254A7C245218C7
:10302000A33214709A79DC79825C144207D0204C68
:103030005F226418251CA235A1342A7022701A7AE6
:103040005C7A825C144204D0194A7C245218A03263
:1030500014709A7ADC7A825C144204D0144A7C247C
:103060005218503214701A7B5C7B825C144207D079
:103070000F4C5F226418251C523551342A7022707F
:103080009A7BDC7B825C144204D0094A2E245218BD
:10309000A43214701A7C5B7C825C134204D0044B13
:1030A0005918F43127230B70002030BDAD000010FB
:1030B00060130010F8B52D4C071C0025201C2021A2
:1030C0004F22FEF793FC002D04D0221C7C233932C2
:1030D00023701370231C4F330021013519705034B5
:1030E000052DEBD1214B2D22181C38300270181CF5
:1030F00037300270A1209A705A7040005F221A5433
:103100001B481A54A320400019541A4908784978DA
:10311000385C014204D0191C533152330A701A70C2
:103120000024211C381C0134FFF756FF0A2CF8D16B
:10313000114D124E00242B786A78FB5C1A4201D0A4
:10314000315905E03059FEF771FC0D49091A0A3171
:103150000C48043400F0D4FA0235242CEBD10A498F
:10316000084800F0CDFA0520F8BDC04660130010F5
:1031700041010000610100106C000010800000108F
:1031800063010010A0140010E75C0000F0B585B0EA
:1031900001900027FDF750FB6A4C3E1C6A4A7542BD
:1031A000754113687D19012B05D168480D210C224A
:1031B000FDF702FC02E0002B00D1CDE0002303AAC2
:1031C000537023687F210B405C2B00D198E02ADCF0
:1031D000382B00D18EE013DC072B6AD006DC022BE3
:1031E00000D193E0062B00D0B6E041E0212B00D1C6
:1031F00084E0232B00D187E01C2B00D0ACE081E0E1
:103200004F2B4ED007DC3F2B62D0402B62D0392BA6
:1032100000D0A1E064E0542B76D05B2B3FD0502B44
:1032200000D099E06AE0732B66D010DC662B3AD0B0
:1032300005DC5E2B56D0622B00D08DE062E06F2B58
:103240003BD0712B52D06D2B00D085E02DE0792B37
:103250004AD006DC762B4BD0772B3DD0742B7BD11C
:1032600046E07D2B23D07F2B25D07C2B74D135E0FD
:1032700031231370022E4BDD231C083B1B681940C1
:10328000542908D0032E43D0231C0C3B1A687F23FB
:103290001340542B3CD14C2203AB1A7038E032233C
:1032A00035E0332333E0342331E035232FE0362378
:1032B0002DE037232BE0382329E039231370062E25
:1032C00026DD231F1B6819404723232920D11EE038
:1032D00030231CE02D231AE0412318E0422316E09E
:1032E000432314E0442312E0452310E046230EE07C
:1032F00048230CE04C230AE0502308E0522306E068
:103300004F2304E0552302E04E2300E049231370CD
:10331000ADB203A8291C0022FDF7C2FB23681A06E0
:1033200005D5E91D89B20A480022FDF7B9FB2368DB
:10333000DA0572D50735A9B206480022FDF7B0FBC1
:103340006BE0C046F0140010700100104E39000010
:103350003A3E0000EF5C000023680122134206D0D1
:10336000A818C0B2002107220223FDF705FB23683D
:103370000222134205D0A81DC0B200210623FDF78A
:10338000FBFA236804210B4205D0A81DC0B202221B
:103390000623FDF7F1FA236808210B4205D0681CCB
:1033A000C0B207220223FDF7E7FA2368DA0606D542
:1033B000681CC0B2042102220623FDF7DDFA23684F
:1033C0009A0606D5681CC0B2002102220623FDF72A
:1033D000D3FA23685A0606D5681CC0B20421072216
:1033E0000223FDF7C9FA23681A0607D5281C0930FD
:1033F0000222C0B20821131CFDF7BEFA2368DA05C9
:103400000BD5EDB2281C0930C0B20B210A35FDF7EF
:103410009DFAE8B20A21FDF799FA013604340C3717
:103420000B2E00D0BAE61B4803210622FDF7C4FA92
:10343000194D1A4E1A4F0024019A2B78D35C6A78E2
:103440001A4205D0A3009859395D0922FDF728FBDF
:1034500001340235092CEFD1FFF738FA002814D0D7
:1034600006240321201C00F0DFF80321C5B2201C34
:1034700000F030F9281CC9B2FDF768FA092C01D117
:103480000B24EEE701340E2CEBDDFDF7DFF905B080
:10349000F0BDC046093800006C0000107401001037
:1034A000A400001070B5041CFFF76CFD201CFFF792
:1034B0006DFE0A4B1B78002B0ED0201CFFF7FAFD87
:1034C000074CC8235B00074EE518211C301C503404
:1034D000FEF754FAAC42F8D1002070BD7903001019
:1034E00060130010DA37000008B5002805D0FDF79A
:1034F00082F90748FFF7D6FF08E0FDF784F9054B8E
:103500001B78002B02D00448FEF738FA08BDC046ED
:10351000A605001079030010F15C000000B5FEE77D
:1035200000B5FEE708B50A4B0A4A0B4903E01078DC
:103530000132187001338B42F9D3084B084900223D
:1035400001E01A7001338B42FBD3FCF725FFFEE745
:1035500000000010485D0000980100109801001064
:103560001C15001002B4714649084900095C490065
:103570008E4402BC7047C04603B4714649084000FF
:103580004900095A49008E4403BC7047002934D0D1
:103590000123002210B488422CD301242407A14225
:1035A00004D2814202D209011B01F8E7E400A142E2
:1035B00004D2814202D249005B00F8E7884201D37D
:1035C000401A1A434C08A04202D3001B5C08224355
:1035D0008C08A04202D3001B9C082243CC08A042C6
:1035E00002D3001BDC082243002803D01B0901D0B2
:1035F0000909E3E7101C10BC7047002801D0002027
:10360000C04307B4024802A14018029003BDC0465F
:10361000D90000000029F0D003B5FFF7B9FF0EBCB8
:103620004243891A1847C046002941D010B4041CEF
:103630004C40A44601230022002900D5494200281D
:1036400000D5404288422CD301242407A14204D251
:10365000814202D209011B01F8E7E400A14204D231
:10366000814202D249005B00F8E7884201D3401A48
:103670001A434C08A04202D3001B5C0822438C086A
:10368000A04202D3001B9C082243CC08A04202D3D4
:10369000001BDC082243002803D01B0901D00909C4
:1036A000E3E7101C6446002C00D5404210BC704774
:1036B000002806D003DB0020C043400801E0802042
:1036C000000607B4024802A14018029003BDC0469C
:1036D000190000000029EBD003B5FFF7A7FF0EBCCF
:1036E0004243891A1847C0467047C04600B50029B2
:1036F00005D000230139037001300029FAD100BD43
:10370000F8B5041CA30719D1231C04CB0F4D104E90
:1037100050199043021C201C32420FD1181C0B4F31
:1037200004CBD5199543354208D1181C074F04CB5B
:10373000D51995433542F1D000E001300378002BD4
:10374000FBD1FEF77CF9201CF8BDC046FFFEFEFE53
:103750008080808053455249414C20434F4E534F07
:103760004C450025732072656164790D0A00444D53
:1037700031324343000D0A4279652E2E2E0D0A0088
:1037800025732025732025730056414E494C4C412A
:10379000005633002578000D0A25303278202000AD
:1037A0000D0A413A2000202025633A20000D0A4DE1
:1037B0003A20002020473A20253032780D0A005761
:1037C000616974696E6720666F7220646174612E2E
:1037D0002E2E0D0A00526561642025730D0A004FDC
:1037E0004B004641494C454400656E61626C65641E
:1037F0000064697361626C6564004C4344206465D5
:103800006275672025730D0A00030300000003039F
:10381000005C0003030C000C03037C287C03037C86
:10382000447C030324104803032854080303000CBA
:103830000003033844000303443800030320100846
:10384000030310381003038040000303101010031B
:103850000300400003032010080303384438030327
:10386000007C000303645448030344542803031CEE
:10387000107C03034C5424030338542003030474C2
:103880000C03032854280303085438030300500092
:10389000030380500003031028440303282828034F
:1038A0000344281003030454080303384C5C030347
:1038B00078147803037C5428030338444403037CBE
:1038C000443803037C544403037C14040303384446
:1038D0003403037C107C0303007C00030320403C82
:1038E00003037C106C03037C404003037C087C03CF
:1038F000037C047C03037C447C03037C14080303E3
:1039000038447803037C14680303485424030304F5
:103910007C0403037C407C03033C403C03037C2089
:103920007C03036C106C03031C601C030364544C85
:1039300003037C440003030810200303447C0003BA
:1039400003080408030380808003030408000007C1
:10395000080400000000BF01BF01090500000700C6
:103960000700070007130A00002000E400FC003FE6
:1039700000E700FC003F002700040F0800000C01D6
:103980001E01FF03FF032201E201C2190D00000E18
:10399000001F0011019101FF007E00FC00FE0113D9
:1039A000011101F001E0140A0000EE00FF01110115
:1039B0001101BF01EE00E00130011001050300001C
:1039C0000F000F0A050000F800FE03070701040BB3
:1039D000060000000001040707FE03F80F080000BE
:1039E00000000A000E001F001F000E000A1109004F
:1039F00000100010001000FE00FE0010001000106B
:103A0000080400000004800780030D070000100078
:103A100010001000100010001008040000000080CA
:103A20000180010D07000C000FC003F0003C000FE7
:103A300000030F080000FE00FF0101010101010168
:103A4000FF01FE10080000000002010201FF01FF5B
:103A50000100010001100800008601C70161012179
:103A60000131011F010E010F0800008200830111C6
:103A70000111011101FF01EE1109000030003800B1
:103A80002C002600FF01FF012000200F080000800D
:103A9000009F011F0111011101F101E10F08000058
:103AA000FC00FE010B0109010901F901F00F0800FA
:103AB0000001000100C101F1013D000F00030F08EA
:103AC0000000EE00FF01110111011101FF01EE0FD5
:103AD0000800001E003F0121012101A101FF007E1D
:103AE0000804000000008C018C01080400000004A0
:103AF0008C078C0312090000200070005000D800D1
:103B000088008C01040104011109000048004800EC
:103B100048004800480048004800481109000004D7
:103B20000104018C018800D80050007000200D07AE
:103B3000000002000300B101B9010F0006190D00D9
:103B400000F800FC010603FB06FD0505050505FD63
:103B500005FF050601FC01F8120900008001F001D3
:103B60007C004F004F007C00F00180010F08000036
:103B7000FF01FF01110111011F01FE01E011090008
:103B8000007C00FE0083010101010101018301822B
:103B900011090000FF01FF01010101010101830181
:103BA000FE007C10080000FF01FF0111011101114E
:103BB00001110111010F080000FF01FF01110011A7
:103BC000001100110001120900007C00FE008301B9
:103BD000010121012101E301E20112090000FF01BD
:103BE000FF011000100010001000FF01FF010A0586
:103BF00000000101FF01FF0101010B0600010001AE
:103C000001010101FF01FF10080000FF01FF013861
:103C1000006C00C6008301010110080000FF01FFD5
:103C20000100010001000100010001160B0000FF6E
:103C300001FF010F003C00F000F0003C000F00FF0E
:103C400001FF0112090000FF01FF010F001C0070BD
:103C500000E001FF01FF01130A00007C00FE008369
:103C6000010101010101018301FE007C0F08000038
:103C7000FF01FF012100210021003F001E140A0066
:103C8000007C00FE0083010101010101038307FEA6
:103C9000047C0412090000FF01FF012100210071D2
:103CA00000DF008E010001110900008E009F01114C
:103CB00001110111011101F301E2110900000100DC
:103CC00001000100FF01FF010100010001110900D5
:103CD000007F00FF008001000100018001FF007FE4
:103CE0001109000007001F007800E001E0017800E2
:103CF0001F0007190D00000F007F00F001E0017C9C
:103D0000001F001F007C00E001F0017F000F12097E
:103D100000008301C7016C00380038006C00C70147
:103D2000830111090000010007001E00F801F801DD
:103D30001E00070001120900008101C1016101316B
:103D40000119010D010701030100070008000A0124
:103D500000181110133831303378717073C8C1C036
:103D6000C38881808384848782C5C4C7C275747701
:103D70007235343732151417120207020802010097
:103D800003010903040204020503050006466972E3
:103D90006D776172652025735F25735F56330D0A59
:103DA00000436F6D6D616E64202020204465736355
:103DB00072697074696F6E257300252D3130732020
:103DC00025732573000D0A5479706520273C636FB5
:103DD0006D6D616E642D6E616D653E203F272066BE
:103DE0006F7220706172616D730D0A005570746995
:103DF0006D65202575730D0A003F0025730D0A0DB2
:103E00000A00564F5941474552203E3E2000256347
:103E10000048656C70004E6F20706172616D7300B8
:103E20004B6579207072657373003C6B6579313E28
:103E3000203C6B6579323E202E2E2E0044756D702D
:103E4000206D656D6F7279006C004C6F6164206D40
:103E5000656D6F7279007400546F67676C652064DC
:103E60006973706C6179206F757470757420746FEC
:103E700020636F6E736F6C6500000000008001505E
:103E80000080025000800350FC3F0150FC3F025074
:103E9000FC3F035025735479706520273F27206627
:103EA0006F722061206C697374206F662061766187
:103EB000696C61626C6520636F6D6D616E64732502
:103EC0007300074E7038EE4FE5004EE06E146BA99C
:103ED000003B1860EC11E8F093E42E20305ABC70DF
:103EE0005942E500E52C664F9D4E9C3BE52C6660F3
:103EF000E03B17B876F84C817B47287140B0A8AEFC
:103F00004404A0951C2D44D41304700CA90C0C215E
:103F10000B5C0635584C178CBD2C44604E706E28D7
:103F2000600014735C6106B08C77BB4E48A34518E3
:103F3000F0E01624451B4D35CB7A9960A0C92CCCF6
:103F400060CB140BF4FEC99C53DB334370AEF0AE70
:103F5000E09481068C215B601110F3D45B1C53AE9E
:103F60004E7038AEE04E70389C735D4C4E70781CCD
:103F70003B5D4C4E70B89CEED8F8D4CE14EBFEAE40
:103F8000D8E0151E46FB4E4F1B893094E38CB536A6
:103F90005344D8589502666666E6E65C6354339CE3
:103FA00098D84C77486B54879CE3546F9C63543F7C
:103FB0009C8B54379C6394635C53141B5C14F35CBC
:103FC00014D35CA394FB5CEB941B5CAB5C949B8C68
:103FD00007E95A145B5C66666666666666666666D0
:103FE0006666666666DB94255B941F5C6B1C84E6E4
:103FF00045025C06D3DCEB541B9CA354CD4FD41B71
:104000001C9B1413885B6666666666547F666666EC
:1040100066545B30EC06F6F656868646CB941B5CFF
:10402000AB1453421F664BA28CA5175B66E61413B4
:104030005CDCA6D4EB84650A946BBD36946B9CD88B
:10404000D8487B30E09417661C0263940B9CD8D848
:1040500044D8D8B0E33006064F300B062B54AFD40B
:10406000BF94231CD01B94231C10DB54231C50B37F
:104070001C909B30E146A330DCE394235C5906940A
:104080000B59401C06EA6786A222CA531110B12CB4
:104090009502624B2690A88CA3B51C33E662C34AF6
:1040A000B38CC748B81CEA1FBD2C1110B12CCD40F1
:1040B000D8AE4C13112C98FD1CF3112CB51CE360E9
:1040C0000C2F084C27FB112C043BAD2CCC495BCCAE
:1040D0002BA9008CA3F51CF13C45128CEB8EAD2C6A
:1040E000CCDFA8F51CCC134E1C6EEE2BEEEEDCDC08
:1040F00076DB6A1427D4D46AEEF05502762B5CCDB9
:104100004E488C8F060C1720B0611C1C6223EADC21
:10411000E3A2140FD4274C177E8ED4D4AAEE3CDC35
:10412000CABCAEEE5C1EA05A970EAE6E5B8C1FBE74
:10413000C70CE7FA3102BE44F0DB427FA6FAE32661
:10414000C3E68C130C035CB0EA8EA09C8A8A8A8634
:10415000061CD62B8A538A06AEFCAE261C5E2FA602
:10416000EE8ADBA66E2D4454F9026BE930DB9CA28B
:10417000A2A2BB84488C7F611C2E5C22029C6A0830
:104180005A4F046A33FA6BEEDCD0EE3EF30CE72EA6
:104190006B7540F6271CE257FA43FE37E0BD40FA44
:1041A000A09CCD4E8C60CCD7C8E04940F895185DF6
:1041B0004C494038BE792959545D4C195079285DD5
:1041C0004C251CA9004D18FACBC500F11CFA4B8DEB
:1041D00000DA4B951CFE5B5950BEEF0E98BA792859
:1041E000BB8D00051CA900FD404D18FAE3C500F188
:1041F0001C8D00951C59501D44FE770E4E5C50508E
:1042000050663D19D940E8E30150CBC550B00102DA
:104210009D5CED18BD00251CE9188D00DA7B5D1C46
:104220001D4428F0A13CB04433513C1D4468ABCD43
:1042300040A95CB8FAFD401D1CED18E118E9181DF5
:1042400044BEE803133373C38382C2723212103048
:1042500070C08087C7773717113171C18184C474EA
:104260003414183878C88884C57535150E1C9856CE
:10427000C6AE1E585C5ED4A6F31467F6C7661B066E
:10428000C31417D43EC3985E1CF6138A9C0EEAEA48
:10429000EA081C93068E26F32E8A6E2E5A5F5E4F16
:1042A000FA2F5E5F1E60AAE00A4EC7D46E5B3ED452
:1042B0008E9BBC88E4E8D8787CA8FCF844404CF499
:1042C00074823F48B3266B16FD316935A934E81175
:1042D000491246134E146D1519215122642371247D
:1042E0001D255E481A208B306A108D4077342F11BF
:1042F0008912E113B614001507210922E523E424ED
:10430000E3259A48642671169431A6359F34AE1180
:10431000B512AC13BC14D015F321222275236F24DF
:10432000762508F024F139F22CF3043600361AF61B
:1043300035F738F868127C14E03157336E325D156A
:104340006311F849F94988AED8C4F51CF13C4E7A9E
:104350008CBD1760164E7A5C10101C90064517C66F
:104360008C77300B0653300606370CF512CD4030F3
:1043700042068B8E4E1A9C10300BC61F5AEB4E1CF9
:1043800010CAEA8C4917BC30064E3039BC705AA6A8
:10439000BC1A7030036E061F951CB0A0E0A6C13891
:1043A00038AEC31C3042CA3005CA5B4A8C231C227B
:1043B00053F538C116CAB34A8C3BBC1C505003C6D7
:1043C000F538B048082D44D43FF00102CA3B4A8C6E
:1043D000B35C1043CAEB4A8C535CD03C30F006BC53
:1043E000BD166D10BE1F6D103D182D44D4B1361C86
:1043F000CD4ECA634A8C235C90136D10851C638C70
:10440000235C50C36D10B91C138CFD0A4E6EEF1C5B
:1044100090BCCBA606629F62638CAF1C98A258F337
:104420001C9006C362D38C4B1C50BC1CA27CBD16D6
:10443000B93838F0A13CB0F90230EB7D3C9502620E
:10444000538C47B938B044040D16626B8C431C5032
:10445000D010103CBB7538DB623B5C8CAF753833D9
:104460008C4B5C10D0D0D0D0BC2BA63007E61CB84B
:104470004AA0A62304A83B0C1BA6DFA62390D0B31A
:10448000606A6066A08AE32AE6A206E6E660B616DF
:10449000F10AB61326BC309C16FC5A7A7CA6F6F6B6
:1044A000F637F67310905BF633A65C105013A61027
:1044B000D00E469CD0EEB8061CEA8B9C226F1CA244
:1044C00086669C23A0266022E3A066A63CDCD0DCA6
:1044D000AAD00E2260609C2260BEE079285D4C3933
:1044E000400EB05EBB06BAF633DD36E6EB66EE5A3A
:1044F000DFE64FBE1EFEFE1EFE138839405E954865
:10450000EE4E70380E7828B868EEE04940F8791C15
:104510005D4C3540382B494078AEF87D1C5D4C35FC
:104520004078C34940F8BE0E784349407928D349C2
:104530004078791C5D4C49400EB8851C4948BB1930
:10454000501BCD4079284E1B4EBE5C503BBE00F93F
:10455000182E7A58463E5ED81CD4763654E3EEEEDA
:104560006BD86EEE4B2687D86E26DFAED80E23D8DA
:10457000AE2BD8AED86E9E5E5B8E1E263BD8FCD886
:104580006EA66E264B66CEBE1ED4D4C34EAE98EE3B
:104590002E767676AE5898FE1B66CEAE5C4ABFEE9F
:1045A000AE5C0EE66B3A5BC62622DE6EFA604E1EED
:1045B000E0C6C36E63424F66EAE3A9005B59545DEF
:1045C0004C1154494078FB494038DB4940F8BB98CE
:1045D0009BB09BAE2EFA0E4E5C506657F9182B75A9
:1045E0000066662E7A58463E5ED8065E139E0ED84A
:1045F000DCDC8E132E62F354CB98491AAE9BBE6E50
:104600008E588E4E27980EE026CB5C626EF34130BA
:104610001046F379284E585C50EEAED8AE0B584693
:10462000CB45188D00A375002EFAAE7BFA9BF918C6
:104630002E7A537500FD403D1838666658463EFA9E
:10464000DD36D8465E139ED85EAE6E2E2BD8EE6653
:10465000D85C4E13228EF32EEED4D4D3AE98751AB6
:104660000EBE851F49405846FAC5369B588EEEEE61
:10467000EE0E6ECEEE2798AEE066CB8ED8264B5966
:1046800040A61CE68AA688E63B84666216B670AA37
:1046900038E0F89C4AFEA03C26E0608C60A13C8893
:1046A0001A1EBA044E04E044844484C484C4BB117A
:1046B0001035585C3028C8CC590266DBE07CEEEE41
:1046C0004EE0CD4004A540A80484844E286885406F
:1046D00098AE8C5F851CFA5388FE1BBE082868B80C
:1046E000E8B8CC970918A86D403D18EEF8A140AE87
:1046F000DEEBA838FA3BC88C83F809180522851C24
:104700000CFD4138B1008CDFFE1B88B3BE0E783D36
:1047100018FE7B3853A918A8FEC338FA9D2A8C1FAF
:104720009CFBFE477540D8A54098A84E2885403888
:104730003D1828B80918A8FEAF385540451CE81C9C
:10474000CD4EF8554046179A9A9CAA5CAAA89D3C63
:10475000A54084A8F04EE8688540351C78B10085F6
:1047600040AEA918551CB04518D815389140351CD5
:10477000D81538A140351CF8B1008540B03D18F07F
:10478000B80918A80E8C57F8D85940AE5C0AEEE666
:1047900017DAAE1A131BB0E8754098A888A54078C0
:1047A000284D2248CD4075402138F518049D3C2302
:1047B0006D403D18FE03B8A14038BEB91DF0F80E9B
:1047C00078B91CB045184D1C5D4CB80E78BEB91DAB
:1047D0008D48445D4C48BD2CA084A1009C225D4CBA
:1047E0007540AE4C1F4EA8EE1C8A461FEA8EA540AF
:1047F000F89C0AAEE8CC852B09389140CCE34C6F8D
:10480000A900FD406D407D1C7140AEA8A54009384F
:10481000EEA9007D1CA10025264D4CA9008D48F075
:10482000C500951CF6A3E6977676F673A64CA50F01
:10483000C50019181D44A8F522BD005D4C1918FAD1
:1048400043C500F11C5D4C3B093891404D4C093883
:10485000BEEE8D008D1CC5004D18D85D4C4C5F0917
:10486000389140351CBEAE6D40AEA8B0851CB8B1C5
:1048700000C5005D4C093891406EC5004518A10087
:104880001918FA5B49485D1CABC5005D4CE349480B
:1048900009389140AE680918788D1C551C5D4C098B
:1048A000387928513C6D40B100A540411CA9180E33
:1048B000FE9526A9004C9D0FDA536D40711C59409E
:1048C000F845184A5050A606E633460E8E7A6346DF
:1048D0002F7A1AD3B330104617488950BE1EC954D8
:1048E0004C59268D0019182626001D44A8195489F4
:1048F0000ECD40BD2C3940B0E859086D08494078CC
:10490000D9286838D928284EF0A13C4EB13C19501E
:104910004954D928EE0C2FF8FA172E383540EE28D6
:10492000AEE8BEB03D1870380EF83D1828F9183DB5
:1049300018B13C387140991868F80918E83940F8FE
:10494000A918E8CC1FFA47A900D116A13CCD40B167
:104950003CC8494078BEB13DCD40F90244A1185D44
:104960004C4CB5184C2519891C4948991CBD344C30
:10497000272848534540381B0E1C985CAE1417D4AA
:10498000B6E30E465306DCD42766E3534E9B06136C
:10499000D41477A6E32E8A3A331E7E268ED40ABA22
:1049A0002EFADA0EE088C8CD403D08B059086D08EF
:1049B000AD3C7D3CD928B13CBEE8B0A918707D3C27
:1049C000D9283540F83D18010208130439404D2C10
:1049D000E8B04D2CEEF855404E1C5010EEAE9CE069
:1049E0001C7A831A6FAEE8AE664F2A1B52B78A8EC6
:1049F0009B46D5328851305E7140AEE85940F81A76
:104A0000513071403D18F8711CE8BE5541F8265AE6
:104A10007C26263D187140AEE80C6F38491C2D1CD1
:104A20007859084518BE6838491C28B8491CA86937
:104A300030500E383D18E8F8F613840C330401505A
:104A40000823443150F8BD40E819181D1CBE0C6BFA
:104A5000F0B13C7540FA1770AD3C494078BEB101E9
:104A600038E13C28B8E13CA80C1378010260C45935
:104A7000401C6A3B901B2226A8E0064242CBE6E699
:104A8000D65617C8429BAD2CCCA04A6B7D3C4E9CA1
:104A900050105050E05CC130F130EE4D30CE7C0E05
:104AA0005C4AE0765A5CD0D0FC30F65A56E0843549
:104AB00058C8CCF73004C8CC66EBE04E203C06303A
:104AC00018E0693010D0105090109CEB8E9CB8AA62
:104AD000A6A8B8AEFAFAFAFAFA06661E4E9C905CE0
:104AE000E028D0904C27509050E08EB8AA5CAAA83D
:104AF0000E3B662346CA1BE6D70EA0E0CEE360EE6F
:104B00001C98F6F6C7CE0E7CDCCACAAE4A3C1AA682
:104B10004B4EEE27F8E09A4D30CE7C1A5C4A26F1D7
:104B20003046706518E8C87500CD40A5408444C47F
:104B3000AE5C63BD40FA8B1CCD4E793CF918B13C9C
:104B4000AEE0CE8C1FCC3302275CC8022930453C36
:104B5000F93C5D3C8C2B84913668B08C13F8FEC711
:104B6000C1305CEA9FF1304E9CD04CBF9C1A2BBAEE
:104B70005C0A5C504E2930893CF93C5D3C01308137
:104B80003CE83005465A41300130AD3C6930509028
:104B90005050813C69307D301C109050B91CAD3CA8
:104BA0007C0E2930893CF8813C0130813C69301908
:104BB0003CB91CC1309CA13010101A43B87A1C4279
:104BC0003D3013F93CC1309A9A9CA13050105C1AC8
:104BD0002350502B10D09C501AF1316669180E8C5E
:104BE0007F75003D3088CC5D330EB0C53CFD32CCC6
:104BF00083B08C13F83D30793C488C60E9307932D1
:104C0000D8F918F8714098F09C62A84E5CD0B91C95
:104C1000BD400E4ED0851CE61FFA17D07C0EB0604A
:104C20007EE617CE5CD0A2DC500E040C3D0253B0E1
:104C3000034E1C505C220ED0EEB8D6A03A60B6E30C
:104C4000A05AFC1C02901A3A5C50D01CD0D090D0D4
:104C5000DCD00EB52C2BA90C25581C1066FBCD40C2
:104C600063BE75013D18FE2BFA1B112C95024E9B5D
:104C7000B540B0851C0516B540B8B0E91CC37540F9
:104C80000918EECE2138B0F075404EEEE80138EE4E
:104C90004E93F138EEB0FE4FA538661B46DAE62398
:104CA0005CCD4E5CAADC4ACFAAEEAE7CB6F3F0D166
:104CB00016FE1B1C6B79285E1B9C3B3ECE6EEEEEF7
:104CC0000EEE5A0EEEE613BA4E9C4217AE8E4E6EA4
:104CD000DC50CE5322CEF34EEE947D1BD4CABB865D
:104CE00030E3461C62B8C676C60A7936A65670E02E
:104CF000AEC61C900E3007C25B42A28B30E683A684
:104D00001C90A25F411C23A540B8FEFF661B46DA3B
:104D1000DCEAC7300855405A5E3ECE36CE6066A00B
:104D2000DAE360466BA6061C427F300A4A5B300617
:104D300043E6F7301D06300B1C6262703813754075
:104D40002138603009C69CD0E6C61C13268AF32A97
:104D50001C907038AE1C909C2BAE7CAE766ADBA0AB
:104D6000E01EDC0A5C421FFA1366AE5CC8EE2BC480
:104D700062EE1322E0B028CD4044113C6ED93CAE27
:104D8000F0986EE7A01C100626E630187CBA233A8D
:104D90007A333046DB26CB86460F48113C6EB0CEC8
:104DA0004E3A30F3A66ECFD93C0E986E9F4E7038B7
:104DB000704E6E68A8CCA084A9024E26263C234ED5
:104DC000E34E5CF0CD4EA0D93CF0F0D8D8D8D8D87E
:104DD000D8EE6ED93CCE4E57584E300770EE384E56
:104DE000AE4C9F2EAED8F04E38D8F030E0AEEE6626
:104DF000A06E6656438E006BDC50D4F34CA0EEE000
:104E0000B85C4AB930193C7BD0104C27909C506656
:104E1000E02930E67D30851CABB89C4AAE51309B12
:104E20002878BE57453C4130AE813C311C7940E189
:104E300040AE383D18280EE0B0FA9379285D4C6DED
:104E400040BE0EF82626B91CFA1BF6F348A5480505
:104E50001CF8BE45195EA0930EB0E91C1918FD4060
:104E600093B07140BE3D19FE1FA0E0F8CC5B8C4FA3
:104E7000BD40F845182801181D1C5D4C7540E13CEB
:104E8000B0BE451911183D1CFD408D004D18494814
:104E9000F11C5D4C85184948951E4E70F068A8308D
:104EA000E09C600E290022EBE0B04C6013B0584E3D
:104EB0007078A84E7038689828E00E3D1A3CB6F31A
:104EC000A6E04940B8FBB13CA9023540F8AEFAC5AE
:104ED00036B91C4540354078E91CF90249407879DB
:104EE0002878911CC51651185D4CB0AE4940851C00
:104EF000F83D4CB518B94C4940789B314CB0AE499F
:104F000040851C783D4C5118B94C4940F88D1CE93E
:104F1000184948991C891C3540AE28314C25185138
:104F20003CBD345D4C51184948991C2D44B13C3866
:104F3000E07940691A4940F8794098D44A7D1A8C42
:104F4000A0BEBEBEE045181B3D182D44F05CE049F4
:104F5000400EE02D440E4C1FAD3CAEB13EBE0E499E
:104F600040F8E01538D801387D380E39404EE04E13
:104F70005C509026534E70DCD010901010D0101062
:104F8000684E5C1010D010D01090A8E02030530E66
:104F90004E7038E030E0DB0E30F070B8E04940E3AE
:104FA0002EFAAEDCCED86ECEF66026E63B66EE1E5E
:104FB000D44ECF66E07540BE0EB8851C0D1C4ED099
:104FC00090CC17509C10E91C2BEE4940CEFA174E9E
:104FD000A05CF6336636761B26E0F61B4E2B4A6A3B
:104FE00056D4D4E0792884045E13081E1A6ECEE6E7
:104FF00073CE5E7FDCD494F54726DB0D44D3D144D9
:105000005C336E66AE333A8EF32EEE66AB9CE22BCB
:1050100062E2A7225C53228EF32E542FEE66D4EE6A
:10502000DBAEFAAEE2134E5C6A0E1C500C13A66E99
:105030000E4C3B5D4C1918C14C8C1BBE1EC51AEEA4
:105040004C2BA91CAE6EDC909CFAE3DCE22B628E4A
:10505000587B268E7EA3463C626E0E0C4D1D9BAE89
:105060007EF32E7E983B6E5A5E0E0C1BF11C4C1B81
:105070005D4C11182BEE5C90D010905010501050D9
:10508000905050100B4E54977A103AD4DF54371486
:105090007F94BF54E79CD05C6B9050D05010D050A0
:1050A000101050905CEEE0D0501050D05010101006
:1050B000D0D09C931CD0D0101050D03068DC3B5C1A
:1050C000D0D0D01010D0505CEB5CD0D030311CB3BD
:1050D00030339C934E70EED8F81A9ABABABA1CEADA
:1050E000E6E838EE7828B868BA463CFED813FE6F7A
:1050F000F65F0E8E1CEE8A5C4A23A6C39B66061BD7
:1051000036E04E22CE3EEEC21BAA260EC223EE2E63
:10511000FBDE338A6E262EFB6A626B7E5BEE865A5E
:105120005E2A4EBAE0481B792848DA7F4948FADD02
:105130003698FEE72EC51A792844043E5E97DA8336
:10514000A606E67B461BA6080E5E5A5C8A62228E85
:1051500058B35CCE62AE4E254E422766EEE3D825AC
:105160001CB31118B344043EAE2B44042EFA0E2691
:10517000E68B5E57AEF51C5C4EA60E6E3B08CB541C
:10518000FFD43E26DB538E7EF3982EBE314A3E6E10
:10519000EED49493AE8EEAEAEAAE9CD086C6E35C87
:1051A0008EEE0D447D4CFAE3D4BB2E9C822E8ECD28
:1051B000440C376E8E6E2E6E1C7D4CFA3B8EDBEEF1
:1051C000DB8E235EEF665E0C1BBE0069184CCB497C
:1051D00048951C98FE9546A6EEDB8EA91C6E5C1BBE
:1051E0002E62F34226DCE08CA04ED8D144EEF11EB4
:1051F0004E66A02660A6E33C013EA01C109C5020F9
:105200001378EE68A886BD2C4E5C906E27CCEB30F0
:1052100082065ABC3006203C5666B76E66302806B9
:105220000F4E6E1C50903158538459401A352C46FD
:10523000707A7FBD2CE52C30126603843017666BC4
:10524000307566A3301466D32666AF88BD2CCD3882
:105250008CEF1CE02059029CD806308006D8B02183
:105260005A089C304258613C30F0292CA8A0706E3E
:105270001C5090D06B5417844E04606ED436D4EB1F
:105280001C9090901090BCDCD00EA01C4502B5186C
:105290004BBE45192BAEBE79294E7078A83868CE22
:1052A000BE1E28F8BA9CEAEAEABAE8AA8A8A8AE024
:1052B000513C4E7038BE5CEA28F89CEAEAEAAAA69D
:1052C000E85B9D5C5954151CC14C251CFD40C9541C
:1052D000115489501D4468E0FD405E1BF67B8D48EB
:1052E000A1008D488D00F11E849C98D84C1FD8E0F9
:1052F000D888E025545D4CDA99513D08F69BBE09EB
:10530000190D1C8C13A0F84518513CFE4152C88859
:105310000E4E9CD0064B44F15456231C621F4EA8DF
:1053200059407C463CA8BD2CCD404885545D4CA0DE
:105330008554E954A95451547540E62762623FA947
:1053400000F154DA87CD407B30E070B86666FEA08D
:10535000F6607D0A5D1C5D4C1918151C515459549A
:10536000E11851542554DA9B4D548C3B7540BD4097
:1053700081545D4C2554513CE1185D4C51542D54E1
:10538000DA8BD154DAE34C9D3C444875408C0118CB
:1053900070A0C14C3D1CA954CD407059543D1CC552
:1053A00000951CA954B0A918E118BD00B0FD4045F6
:1053B00018F154DA474948EE98511C2B5D1CE91846
:1053C000151CA9544D1C5D4C2D54D154F11C489D05
:1053D000484D54513CF1544D1870BE62EE33594063
:1053E0007CC63CA81950AEDA2626A8B0CCB7BE3D84
:1053F00019FA8BB0FE1FF6134688466666F6995278
:105400001C22E7B02626A88470A90275408C237858
:10541000792ABD400E78851E75408C1BA043BD4087
:10542000A918BE49550C1B0C6038451A4940F8793B
:10543000280CA00CA0A3AE583940F80EF873AE5853
:1054400059407C064940B8AEBAA6A6EEE0AE58591F
:10545000407C06F81EB3DAA05EBFCC890988C42D53
:10546000544D185940CEBE1EE8B87CA606BCA8E034
:105470008C23CC8908FD40D1544D18C83940CEE862
:10548000F8BAAEE80EE00C99517540BD408CA719F2
:10549000508D1C111AF154E30C1B0C605D4CF51877
:1054A000513E4479285D4CF15448914AFE2D54FEFA
:1054B000D1555D1C49484D185D4E883940B0287162
:1054C00040F84C1778F54019403940380E851C4992
:1054D00040384C17B8F5400D4039404C1F48030E7A
:1054E000B0851CF5404940780D400E62F5404940BA
:1054F0001940F0A8F0A90204010208EB613C5940F0
:10550000C676C61B290062EBA0F08459408C33C6D6
:1055100076C6292C1C4AA8190AF918A8AEF902F176
:10552000387D38C516B540E91CD3B540B8851CA3F5
:105530000E9C30E5290062EB4E707D3C9502754073
:105540002138F0A13C7540A918B1365C481B0E44C7
:105550006084395C4E70E0AE28FE1BFE4F0C3B9C15
:10556000E21FD013D0A83C364F852CD61B5C903C54
:105570004EB83C3657852CD61B9C107CF11CB83C91
:10558000364F852CD61B1C103C4EB87C364F852CD4
:10559000D61B9C10FC4EB8BC364F852CD61390FC05
:1055A000F11CAE655C0EB87C3657852CD61B5C9022
:1055B000BCF11CB8BC364F852CD61B5C90BC4EB8D9
:1055C0003C3657852CD61B9C103CF11CB87C364FC2
:1055D000852CD61B5C10ED1CB8FC364F852CD61BD9
:1055E0009C10FC4EAE315C8C234C0D5F1C98F64336
:1055F0004E3008A8300C3B4E300CA8300868A0385C
:105600001E7EB77E8F7E3BB8BC4EED1C63A0BE6095
:105610000EFC9C0278A297A20FA24FA27FA2F7A233
:1056200047A26FA2EFA22F637C4EB8ED1C6EB87C30
:10563000F11CB8BCC3B87C4EE37C4EB8BCF11C6E08
:10564000B83C537CF11C6EB87C4EB8BC4E9CB0FE8E
:1056500023109C427870686E5D5C4EA094233001EC
:10566000BC942330001B14E7E00C1F1C10255C4E7B
:105670008C1BDC501C98F6F61F5C10F6F61B1C50B9
:1056800046595C695C38EEA0E020E00E7870686BEB
:105690004C60C8CC6088C92E0EB870A88C9BCCA07A
:1056A00048E04940B0A8448922CD40BE4879285DF1
:1056B0004C195048A548C14C1950FAE91FCD40FD7E
:1056C0004200A1160840413038353113356F155569
:1056D00008E20C8028C208368B0A1670A2E25565D3
:1056E000C8BC052029727028B283300683C560517A
:1056F000EFD01565D52113D5B3CDCC1E1E5E5E75DA
:1057000096241103512C485555555505F41C328BE0
:1057100023D0CF55711584D507D44C86D0F239806B
:1057200081730474E3DC504C8C40ECF0C7BF47C677
:1057300011D09C8C231362FF7CF3FC2232123709B8
:10574000332B8EA3420CB88C3C020B30F0EFCC8391
:10575000E24886CC107F24111F72700E805819CA3F
:10576000DFC39A30F2C3D280C4F4030CC620AA0C63
:105770001BF4B1636CB2C8227238F2EE63CCECCC8D
:10578000C80C88A88489808014838084A8840080C1
:10579000C69A120300312310A20133F8C0C76CC0AF
:1057A0004C800E000000000000000000D03034F7F4
:1057B0008880ECB1487FC20E34E393CDCFFE511404
:1057C000059122122032332333333532526664740A
:1057D00067668A9899999999A98888A880A8EAFE05
:1057E00062EE199332D8085A7B3431318FC40114D8
:1057F000D1183D1D5190053338001F4534094434FC
:105800000C053890114D114D10362323C02CD1C4F6
:10581000034F38F1810450C70FB01D53CC03304003
:105820004CC4030E31752A183D3C059C048FE14A97
:1058300047AF6A37BD0C6C9B3815110416441CB376
:105840002C7363BA8183B97ACF4C0CC8B8BF502986
:105850000E0112000F325203C8488C76330C3213FB
:1058600000083180830004F4F958D8C4D304118DA2
:105870004D464CD30E914A49F3C085A0E030F3FB6E
:10588000D2CCCCCC8C040071028842408AE4937F55
:1058900043424FED47100C0D44B1C80220004808A8
:1058A0001A3829064CDB60F74E9330E118942C71BE
:1058B0009B0E3F490AC285EFFA084D43928B5C1F4D
:1058C000BED5B2545012048258552489B0A06564E4
:1058D00022501421698966A409252E49912425792D
:1058E0000323CD7CC8230525500801482150081406
:1058F000829054D520CB8C2C9D942C12F124E24B19
:105900000655203195118F5332230CCFF352D1100D
:10591000222331212C8184CC482020A1C22102875E
:105920008C88C41032210222CD85800C03874C085C
:10593000222202810C104212C0C4CC844C24C861C3
:1059400013B34014040C7FC8603388287084CCD013
:10595000CC2C2FC33012022C3C04201412C824F18A
:10596000F2148D42CC0CB333400C4108C8402C9D3E
:105970008CDD454B03B13404F90074C83033222365
:10598000042283C43C03034306D20C13F1F54120E7
:105990003C172287CE828AF00CF0880F0F032D2E41
:1059A000CC30C6B180C38830B3F1FC3C87CC12FA4E
:1059B000D5DFC0C23CB0FD0000080BECC0CB1FEF30
:1059C00023C550527341F13FC17C34D187D4C248C2
:1059D000CE3235CD83B2D60008020E8848CB85275B
:1059E00001C3878C0201D141000A2810DB04130493
:1059F0000444210101400150144110050444404079
:105A0000930003BC408F622038854448840040C422
:105A10001C1224417211118864A8CC781B11AEC5E8
:105A2000992D52FAF6EA0D22EA822222132000C8AA
:105A3000C0221028B0000122C2920C0FDC86F8CCE4
:105A4000032554D8F36063F7F31FDDFB03CE5F74C7
:105A50001DF33E482A8CC680BBD90A3D218146B140
:105A60004A12460763F7820DA33BF04CACA83809F5
:105A700000409727213877770084E5400D06EA0338
:105A8000A8302201143C401F21044442063C726CA1
:105A9000CE9D40009338044002501240C404498D0A
:105AA000CC8CAD219280CA132011A248CF19CB0211
:105AB000238322102210130028C4223E0E2120C46A
:105AC00089CD2313024E8800300D123130C0C40C32
:105AD0000C0C30310304880C4DCC4C80C0F4CC3C11
:105AE000CD30B220E04F43328CCD47220D33384ABF
:105AF0008C2CCA0A3A841C17FE0C48E08AF3BBD8E7
:105B00000010740183E0A2E201C83F360104E3847F
:105B10000F12F4760BA23876B523E36C12128C8C3C
:105B2000D80002862C12EE1015EED540013022036B
:105B3000648816638295D54442213503A4041D6010
:105B400014072029D0D98A54FC415105D022C13FE5
:105B50005DE3B8C812779C8DFB40314C024ECE4CB1
:105B6000F14E12069C5223C3F809620105D9030CB9
:105B700041D7BA7B25F20C3FA73503E24C4B10010D
:105B8000C8C3BC844C0024C40B99E33309016A03E5
:105B90005D8C2903F8B774C2523C06D2D3E0CDC461
:105BA000121313E330C2784C2104071373D80E8C00
:105BB000BADEBA791081020E5641453FF13F1853C3
:105BC000FCD033301033001F632222C10C3FC708C2
:105BD000230A40CA281E33C71C3CD113CC241222EE
:105BE000A2484810AEEE1323203112322031133375
:105BF00023A2E18F0B42031304080C314248081022
:105C00001001132311C44C086A132DA0338A20C23B
:105C10006AB1A30F083CD1201011C6F0320EFF3438
:105C200005343543318DDD3E4C880CF4121F4C8415
:105C30003010D4830408483C3C31CC44A2180132D3
:105C40000C0940C8144C40C80007C4241423481051
:105C50003CB3231ECFEC3303008484C032CC210E2E
:105C600013128CC40C618350442063CBC858CA48BB
:105C7000322123582123492123380C2523C1A48C08
:105C800088958C209332B21332A2C404334114108D
:105C900045555554938A5754455444410D35414711
:105CA000D5D034745548E5321011140EDC303085EF
:105CB00015C14CE0E7C27F93DBCFC34FC88C2423D0
:105CC00046040304050A08060BFF0209070D010C30
:105CD00000FF2025692025692025692D25690020E0
:105CE0002025633A256900202020205F5F7C002C5E
:105CF0000044697370206F66660D0A005553455263
:105D00000046004700424547494E00524144004486
:105D10002E4D59005052474D0055534552202020DA
:105D2000006620200067202000424547494E202081
:105D30002020200052414420202000442E4D592094
:085D4000202000432020200078
:105D4800F93D000000000000610D0000113E000058
:105D5800163E0000143E0000FF000000B9060000D7
:105D6800203E00002A3E00008737000000000000A7
:105D7800A50400003C3E0000163E0000483E00001E
:105D880000000000B10500004A3E0000163E000079
:105D9800563E00000000000011070000583E0000B9
:105DA800163E00000F000000F4010000040103018A
:105DB8000201010411040F04170416011801000060
:105DC800195D0000215D0000255D0000295D0000CF
:105DD800035D0000345D00003B5D0000435D000092
:105DE800145D000000171B243E4253697505020527
:105DF8000804080B08040405010504090809040639
:105E08000807020602040206010604070103080344
:105E1800040C080D020C0203020C010C040D010D08
:105E2800080D040802080807080202070408010808
:105E380004090209010A080B020A0201080A010AF8
:105E4800040B0102080204100811021002110810C4
:105E58000110041101120212011302130812080F93
:105E6800081204130113041402140115021508146E
:105E78000817081404150115041702170119081A40
:105E88000219021602190119041A01160816041B30
:105E9800021B081A0818021A041B011B0418081808
:105EA800040B042020202020202020202000000097
:105EB80001000000FC5C0000015D0000035D0000C3
:105EC800055D0000035D00000B5D00000F5D000034
:085ED80073370000145D0000A7
:04000003000035259F
:00000001FF
